:100000000C94ED020C941C030C9408030C9408034C
:100010000C9408030C9408030C9408030C94080334
:100020000C9408030C9408030C9408030C94080324
:100030000C9408030C9408030C9408030C94080314
:100040000C9499040C9408030C94B5040C940803C4
:100050000C9408030C9408030C9408030C940803F4
:100060000C9408030C9408033B073E074107440720
:1000700047074A074D0750075307560759075C07BC
:100080005F076207650768076B076E0771077407EC
:1000900077077A077D0780078307860789078C071C
:1000A0008F07920795079807494E464F3A203078B8
:1000B00030312C200032303036303632392D31207C
:1000C000524453204465636F646572206279204D09
:1000D000617263204B6574656C20616C696173208B
:1000E00044694E6F2C206D6172634061746F6F6D57
:1000F0006E65742E6E65742E000D0A00423A203033
:10010000782530376C580D0A00494E464F3A20305A
:100110007830322C204E6F20524453207369676E22
:10012000616C2E0D0A0047524F555025303275250F
:10013000633A2030782530345820307825303458D0
:1001400020307825303458203078253034580D0A46
:100150000050493A203078253034582C20446574BA
:100160006563746564206E65772073746174696F6C
:100170006E2E0D0A005054593A20307825303258EE
:100180002C20004E6F6E652E004E6577732E004357
:10019000757272656E7420416666616972732E00B5
:1001A000496E666F726D6174696F6E2E0053706F69
:1001B00072742E00456475636174696F6E2E00441D
:1001C00072616D612E0043756C74757265732E00DB
:1001D000536369656E63652E0056617269656420BC
:1001E0005370656563682E00506F70204D7573699C
:1001F000632E00526F636B204D757369632E00454B
:10020000617379204C697374656E696E672E004C5A
:100210006967687420436C6173736963732E00535C
:100220006572696F757320436C6173736963732EB4
:10023000004F74686572204D757369632E005765B1
:1002400061746865722E0046696E616E63652E008A
:100250004368696C6472656E2E00536F6369616CEC
:1002600020416666616972732E0052656C69676928
:100270006F6E2E0050686F6E6520496E2E005472AE
:100280006176656C202620546F7572696E672E004A
:100290004C656973757265202620486F6262792EFD
:1002A000004A617A7A204D757369632E00436F7539
:1002B0006E747279204D757369632E004E61746996
:1002C0006F6E616C204D757369632E004F6C6469AD
:1002D0006573204D757369632E00466F6C6B204DFE
:1002E000757369632E00446F63756D656E7461721A
:1002F000792E00416C61726D20546573742E00413B
:100300006C61726D202D20416C61726D2021005551
:100310006E6B6E6F776E2E000D0A0054502654419E
:100320003A20307825303258203078253032582C19
:1003300020004E6F207472616666696320616E6E84
:100340006F756E63656D656E747320617661696C3F
:1003500061626C652E005472616666696320616E2D
:100360006E6F756E63656D656E747320617661691D
:100370006C61626C652076696120454F4E206F6E1E
:1003800020616E6F746865722073746174696F6E3A
:100390002E005472616666696320616E6E6F756EC1
:1003A00063656D656E747320617661696C61626C02
:1003B00065206F6E20746869732073746174696F4F
:1003C0006E20616E64206D617962652076696120BE
:1003D000454F4E206F6E20616E6F7468657220739A
:1003E000746174696F6E2E00547261666669632071
:1003F000616E6E6F756E63656D656E7420696E20DB
:1004000070726F67726573732E000D0A004D533A58
:10041000203078253032582C20004D7573696320C8
:100420006973206265696E672062726F61646361DF
:1004300073746564206F722073746174696F6E20C9
:10044000646F6573206E6F7420757365204D532043
:10045000666C61672E005370656563682069732060
:100460006265696E672062726F616463617374654F
:10047000642E000D0A0050533A20002563000D0A37
:100480000044493A20307825303258002C205374EB
:100490006572656F002C204D6F6E6F002C204172CD
:1004A000746966696369616C2048656164002C2029
:1004B000436F6D70726573736564002C20537461B3
:1004C00074696320505459002C2044796E616D6921
:1004D0006320505459002E0D0A0041463A203078CE
:1004E000253032582C200025752E25754D487A2E42
:1004F0000D0A0041463A203078253032582C2054DD
:100500006869732073746174696F6E206861732009
:100510006E6F20616C7465726E61746520667265C1
:100520007175656E746965732E0D0A0041463A2037
:10053000307825303258203078253032582C200041
:1005400025754B487A2E0D0A0025754B487A2E0DDD
:100550000A004C413A203078253032580D0A0045C7
:1005600043433A203078253032580D0A0052542542
:10057000633A20002563000D0A0043543A20307886
:100580002530315825303458253034582C2000552A
:10059000544320253034752D253032752D253032C9
:1005A0007520284D4A442025752920253032753A7A
:1005B000253032753A3030202563253032753A25A2
:1005C0003032752C200054494D4520253032753A83
:1005D000253032753A30300D0A0011241FBECFEF9E
:1005E000D4E0DEBFCDBF11E0A0E0B1E0E4E1F9E28C
:1005F00002C005900D92A630B107D9F711E0A6E030
:10060000B1E001C01D92AF32B107E1F70C94E304F1
:100610000C940000982F8091C00085FFFCCF909330
:10062000C60080E090E008958091C0008823E4F740
:100630008091C600992708951F920F920FB60F92CE
:1006400011242F933F934F935F936F937F938F93D7
:100650009F93AF93BF93EF9340911E0150911F0161
:100660006091200170912101E0910B01440F551F11
:10067000661F771F4C9B04C04F5F5F4F6F4F7F4FCC
:10068000809124018F5F80932401809106018F5F08
:1006900080930601809106018A3191F4DB01CA0141
:1006A000B3708093070190930801A0930901B09360
:1006B0000A011092060181E08093190180931801CC
:1006C000809124018A3129F080911301882309F057
:1006D000E7C07370CB01AA27BB279C01DB01CA01CD
:1006E00081709070A070B070892B21F08BE193E045
:1006F0002827392741FF04C08FE893E028273927AE
:1007000042FF04C087EA92E02827392743FF04C04C
:1007100087EF90E02827392744FF04C08EEE91E050
:100720002827392745FF04C08CED93E02827392777
:1007300046FF04C081E092E02827392747FF04C024
:100740008BEB91E02827392750FF04C086E793E020
:100750002827392751FF04C085E593E0282739274A
:1007600052FF04C083E193E02827392753FF04C0D8
:100770008FE993E02827392754FF04C087E892E0E7
:100780002827392755FF04C087EB90E02827392711
:1007900056FF04C08EE691E028273927CA018070F1
:1007A0009078892B21F08CED92E028273927EE23D1
:1007B000B1F4285D334009F06BC0DB01CA012AE0C7
:1007C000B695A795979587952A95D1F790930D01A2
:1007D00080930C0181E080931301E82F5FC0E1302A
:1007E000B9F4245D334009F053C0DB01CA01072E80
:1007F0007AE0B695A795979587957A95D1F7702D5C
:1008000090931D0180931C01E0931301E2E046C028
:10081000E23029F580911C0190911D0193FD04C0E7
:1008200082E02C35380749F080911C0190911D0120
:1008300093FF2EC02C5C334059F5DB01CA013AE02E
:10084000B695A795979587953A95D1F790931B0103
:1008500080931A0181E080931301E3E01FC0E3302D
:10086000B9F428553240A1F4DB01CA012AE0B6955B
:10087000A795979587952A95D1F790930F01809327
:100880000E0181E080931301E0E08093100104C029
:1008900010921301E0E081E080931801109224018E
:1008A00080911001882359F0419A809117018F316E
:1008B000F8F4809117018F5F8093170119C0909110
:1008C00013019923A9F44198809114018F5F8093BB
:1008D000140180911701882359F0809114018A3105
:1008E00039F480911701815080931701909314017E
:1008F000809117018F3010F0429A01C042984093C6
:100900001E0150931F016093200170932101E09319
:100910000B01EF91BF91AF919F918F917F916F915B
:100920005F914F913F912F910F900FBE0F901F90AD
:1009300018951F920F920FB60F9211248F938091EA
:1009400023018F5F8093230180912301853038F04C
:1009500081E08093180180931101109223018F91FF
:100960000F900FBE0F901F9018951F920F920FB609
:100970000F9211248F938091C6008093220181E011
:1009800080931201809318018F910F900FBE0F90EA
:100990001F90189588EA90E09F938F930E94AB0E6A
:1009A0000F900F9085EB90E09F938F930E94AB0E7A
:1009B0000F900F9089EF90E09F938F930E94AB0E62
:1009C0000F900F900895CAE3D4E0DEBFCDBFC455A9
:1009D000DF4F19821882CC5AD0409924C255DF4F7C
:1009E0009882CE5AD040C155DF4F9882CF5AD0401E
:1009F000C055DF4F9882C05BD040CF54DF4F988204
:100A0000C15BD040CE54DF4F9882C25BD040CD5402
:100A1000DF4F9882C35BD040CC54DF4F9882C45BD9
:100A2000D040CB54DF4F9882C55BD040CA54DF4FD3
:100A30009882C65BD040C954DF4F9882C75BD040D4
:100A4000C854DF4F9882C85BD040C754DF4F9882AC
:100A5000C95BD040C654DF4F9882CA5BD040C554B2
:100A6000DF4F9882CB5BD040C454DF4F9882CC5B81
:100A7000D0403FEFC054DF4F3883C05CD04088E1A6
:100A800090E02EE00FB6F894A895809360000FBE1A
:100A900020936000A89586E090E09093C500809335
:100AA000C4008091C10088698093C10064E173E053
:100AB0008AE093E00E94640E9093160180931501E2
:100AC00081E08DBB8091690083608093690087B16C
:100AD000876087B985B5856085BD80916E0081602E
:100AE00080936E000E94CA04789480911801882334
:100AF000E1F310921801A895809112018823A1F1C9
:100B00001092120180912201873431F4CA54DF4FD0
:100B10001882C65BD0400AC080912201873631F42A
:100B200061E0CA54DF4F6883C65BD04080912201E8
:100B3000823731F4C455DF4F19821882CC5AD04025
:100B400080912201823431F4C954DF4F1882C75B8F
:100B5000D0400AC080912201823631F471E0C9543C
:100B6000DF4F7883C75BD04080911901882319F14A
:100B700010921901C954DF4F8881C75BD040882388
:100B8000D1F08091070190910801A0910901B091E5
:100B90000A01BF93AF939F938F938CEF90E09F9345
:100BA0008F930E94AB0EADB7BEB716960FB6F894F2
:100BB000BEBF0FBEADBF80911101882389F1109295
:100BC0001101809117018823E9F4CB54DF4FB881DC
:100BD000C55BD040BC30B0F4BF5FCB54DF4FB883AF
:100BE000C55BD040BC3071F489E091E09F938F9356
:100BF0000E94AB0EC455DF4F19821882CC5AD040E8
:100C00000F900F9080911701882329F0CB54DF4F6C
:100C10001882C55BD040409B02C0409801C0409AFA
:100C200080911301882331F4E5E0CE54DF4FE8834F
:100C3000C25BD04080911001882309F456CF1092F6
:100C4000100180911C0190911D01892F9927829597
:100C50008F70182F80911C0190911D0193FF03C08C
:100C6000E2E49E2E02C071E4972ECA54DF4FF88151
:100C7000C65BD040FF2379F180910E0190910F0166
:100C80009F938F9380911A0190911B019F938F9353
:100C900080911C0190911D019F938F9380910C0175
:100CA00090910D019F938F93892D99279F938F93F7
:100CB000812F99279F938F9386E291E09F938F9343
:100CC0000E94AB0E2DB73EB7225F3F4F0FB6F89490
:100CD0003EBF0FBE2DBF80910C0190910D01C455F8
:100CE000DF4F68817981CC5AD0406817790709F4C1
:100CF0007BC00E94CA0480910C0190910D01C455E3
:100D0000DF4F99838883CC5AD0409F938F9381E59E
:100D100091E09F938F930E94AB0E9FEFC255DF4FE0
:100D20009883CE5AD040C155DF4F9883CF5AD040D8
:100D3000CF54DF4F9883C15BD040C055DF4F9883BD
:100D4000C05BD040CE54DF4F1882C25BD0400F90C2
:100D50000F900F900F90CE010196CF54DF4F288156
:100D6000C15BD040FC0107E02193015007FFFCCF9D
:100D7000CD54DF4F2883C35BD040FC0170960AE15D
:100D80001192015007FFFCCFAFEFC854DF4FA8838B
:100D9000C85BD040C754DF4F1882C95BD040DE012A
:100DA000A459BF4FFC01BB960FE311921D92015055
:100DB00007FFFBCFC554DF4F1882CB5BD040C55433
:100DC000DF4FB881CB5BD040C454DF4FB883CC5BDE
:100DD000D040C654DF4FB883CA5BD040EFEFC05459
:100DE000DF4FE883C05CD040C155DF4FF881CF5A58
:100DF000D0402F2F332780911C0190911D0165E079
:100E0000969587956A95E1F78F7190702817390745
:100E100009F4A1C080911C0190911D0155E09695A7
:100E200087955A95E1F78F71C155DF4F8883CF5A67
:100E3000D04099279F938F9385E791E09F938F935D
:100E40000E94AB0E0F900F900F900F90C155DF4F87
:100E50002881CF5AD040822F9927AA27BB27FC018F
:100E6000809708F068C0EC5CFF4FEE0FFF1F059005
:100E7000F491E02D099483E891E05FC089E891E066
:100E80005CC08FE891E059C080EA91E056C08DEADD
:100E900091E053C084EB91E050C08FEB91E04DC0E6
:100EA00086EC91E04AC080ED91E047C089ED91E089
:100EB00044C088EE91E041C083EF91E03EC08FEFE7
:100EC00091E03BC08FE092E038C08FE192E035C006
:100ED00081E392E032C08EE392E02FC087E492E09B
:100EE0002CC080E592E029C08AE592E026C08AE61F
:100EF00092E023C084E792E020C08EE792E01DC01C
:100F000080E992E01AC081EA92E017C08DEA92E08F
:100F100014C08CEB92E011C08CEC92E00EC08AED14
:100F200092E00BC086EE92E008C083EF92E005C02D
:100F30008FEF92E002C08FE093E09F938F930E9427
:100F4000AB0E0F900F9088E193E09F938F930E94D8
:100F5000AB0E0F900F90112309F0F2C2C055DF4F76
:100F60006881C05BD040262F332780911C0190916F
:100F70001D0144E0969587954A95E1F78170907040
:100F800028173907A9F4C255DF4F7881CE5AD040CF
:100F9000272F332780911C0190911D018070947040
:100FA000892F9927869586952817390709F461C0F6
:100FB00080911C0190911D0114E0969587951A95DA
:100FC000E1F78170C055DF4F8883C05BD04000914E
:100FD0001C0110911D0100701470012F112706953E
:100FE0000695C255DF4F0883CE5AD04099279F936C
:100FF0008F93C255DF4FA881CE5AD0408A2F9927B0
:101000009F938F938BE193E09F938F930E94AB0EFE
:10101000EDB7FEB736960FB6F894FEBF0FBEEDBF24
:10102000002369F4C055DF4FF881C05BD040FF2337
:1010300019F482E393E00FC086E593E00CC0C0553D
:10104000DF4F2881C05BD040222319F482E993E06E
:1010500002C088EE93E09F938F930E94AB0E0F9097
:101060000F908AE094E09F938F930E94AB0E0F90B5
:101070000F90CF54DF4F6881C15BD040262F3327BC
:1010800080911C0190911D01A3E096958795AA95EA
:10109000E1F78170907028173907B1F180911C0138
:1010A00090911D01F3E096958795FA95E1F781708F
:1010B000CF54DF4F8883C15BD04099279F938F9394
:1010C0008DE094E09F938F930E94AB0E0F900F9052
:1010D0000F900F90CF54DF4F7881C15BD0407723C2
:1010E00019F08AE194E002C086E594E09F938F9323
:1010F0000E94AB0E0F900F9083E794E09F938F9325
:101100000E94AB0E0F900F9080911C0190911D01D9
:10111000E82FE370F1F480911C0190911D0182FF92
:101120000CC0CC54DF4F8881C45BD0408860CC5465
:10113000DF4F8883C45BD0406BC0CC54DF4F9881B5
:10114000C45BD040977FCC54DF4F9883C45BD040C2
:101150005FC0E130F1F480911C0190911D0182FF8C
:101160000CC0CC54DF4FA881C45BD040A460CC54E9
:10117000DF4FA883C45BD0404BC0CC54DF4FB88155
:10118000C45BD040BB7FCC54DF4FB883C45BD0403E
:101190003FC0E230F1F480911C0190911D0182FF6B
:1011A0000CC0CC54DF4FF881C45BD040F260CC540B
:1011B000DF4FF883C45BD0402BC0CC54DF4F288175
:1011C000C45BD0402D7FCC54DF4F2883C45BD0401C
:1011D0001FC0E330E9F480911C0190911D0182FF52
:1011E0000CC0CC54DF4F3881C45BD0403160CC544C
:1011F000DF4F3883C45BD0400BC0CC54DF4F6881D5
:10120000C45BD0406E7FCC54DF4F6883C45BD0405A
:10121000EE0FEE2EFF246E010894C11CD11CF701C5
:10122000EC0DFD1D80910E0190910F016FEF70E0AC
:101230000E945414608780910E0190910F01482FF5
:1012400081878081681731F4FE01EE0DFF1D8281D8
:10125000481769F0CE54DF4F7881C25BD0407530BB
:1012600030F0CE54DF4F1882C25BD04007C0CE545E
:10127000DF4F8881C25BD040843058F4CE54DF4FBA
:101280009881C25BD0409F5FCE54DF4F9883C25B92
:10129000D040F701EC0DFD1D80858083EC0EFD1E16
:1012A0008185F7018283CE54DF4FF881C25BD04045
:1012B000F43009F081C086E794E09F938F930E94F9
:1012C000AB0E0F900F90760107E0D7018D917D0155
:1012D00099279F938F938BE794E09F938F930E941E
:1012E000AB0E0F900F900F900F90015007FFEDCFB6
:1012F0008EE794E09F938F930E94AB0EB5E0CE549F
:10130000DF4FB883C25BD0400F900F90CD54DF4FBA
:10131000F881C35BD040CC54DF4FE881C45BD04040
:10132000FE1709F449C0CD54DF4FE883C35BD040BA
:10133000EE2EFF24FF92EF9281E894E09F938F932B
:101340000E94AB0E0F900F900F900F90E0FE03C025
:101350008CE894E002C085E994E09F938F930E940B
:10136000AB0E0F900F90E1FE08C08CE994E09F93C4
:101370008F930E94AB0E0F900F90E2FE08C08EEA92
:1013800094E09F938F930E94AB0E0F900F90E3FE1B
:1013900003C08BEB94E002C088EC94E09F938F93A2
:1013A0000E94AB0E0F900F9086ED94E09F938F9369
:1013B0000E94AB0E0F900F9021E4921609F095CB8E
:1013C000BB24BB20A9F580911A0190911B0136C066
:1013D000F08A0F2D11271F930F938AED94E09F93AE
:1013E0008F930E94AB0E980125593C4F0F900F90A0
:1013F0000F900F90C9016AE070E00E9454149F930F
:101400008F93C9016AE070E00E9454147F936F9338
:1014100087EE94E09F938F930E94AB0E6DB77EB7DB
:101420006A5F7F4F0FB6F8947EBF0FBE6DBF19C0C5
:1014300080911A0190911B01892F9927F82E8150D4
:101440008C3C78F400E0DE015196FE0131968D91DE
:101450008F1539F0882309F4BBCF0F5F31960B311C
:10146000B0F370EEF71691F48AA58F1579F0FAA60D
:1014700080EE90E09F938F9383EF94E09F938F9300
:101480000E94AB0E0F900F900F900F90B39481E0DD
:101490008B1508F096CF80911A0190911B018A3F1D
:1014A000910509F022CB8BA5282F332780911A01B3
:1014B00090911B012817390709F417CB80911A0165
:1014C00090911B018BA780911A0190911B01892F8C
:1014D0009927F82E99279F938F9380911A019091C5
:1014E0001B019F938F938CE295E09F938F930E94B3
:1014F000AB0E8F2D8150ADB7BEB716960FB6F894D0
:10150000BEBF0FBEADBF8F3058F489E0F89EC0015A
:10151000112480579F4F9F938F9380E495E066C07E
:101520008F2D8051883708F0E0CA89E0F89EC0010D
:1015300011248D579E4F9F938F9389E495E056C059
:10154000113009F05CC0B1E49B1609F0CECAC85452
:10155000DF4FE881C85BD0402E2F332780911A01DE
:1015600090911B018070907828173907A9F080911D
:101570001A0190911B01C854DF4F1882C85BD040FC
:101580001F921F9282E595E09F938F930E94AB0E6E
:101590000F900F900F900F9080911A0190911B0166
:1015A000892F9927829586958770892B09F09DCA86
:1015B000C754DF4FF881C95BD0402F2F332780916C
:1015C0001A0190911B0190702817390709F48DCAF0
:1015D00080911A0190911B01C754DF4F8883C95B2A
:1015E000D04099279F938F938FE595E09F938F939A
:1015F0000E94AB0E0F900F900F900F9076CA123092
:1016000009F01FC180911C0190911D0184FF03C04E
:1016100052E4A52E02C041E4A42E80911C019091B9
:101620001D01182F1F70C554DF4F2881CB5BD040A0
:10163000222379F02A1569F0FE01BC960FE311927E
:10164000015007FFFCCFC454DF4F1882CC5BD04061
:1016500079C0C654DF4F3881CA5BD040131708F0F9
:1016600071C061E4961631F430E4B32E05C021E078
:10167000F22E17C090E2B92E00E0F02E0B1588F480
:10168000FE01E459FF4FDE019C969D91992329F0BC
:10169000903219F08081981751F70F5F31960B1532
:1016A000A0F3C454DF4F7881CC5BD040772309F49A
:1016B00049C0FF2009F446C08A2D99279F938F9334
:1016C0008DE695E09F938F930E94AB0E00E00F9004
:1016D0000F900F900F900B1568F5CC24DD247E0140
:1016E0000894E11CF11CF601EE0DFF1D83A5882373
:1016F00009F18D3079F08A3069F099279F938F93A3
:1017000084E795E09F938F930E94AB0E0F900F900C
:101710000F900F90DE01A459BF4FAC0DBD1DEC0C16
:10172000FD1CF70183A58C930F5F0894C11CD11C8D
:101730000B15A8F287E795E09F938F930E94AB0E5D
:101740000F900F90AE014F5F5F4FE12FFF2721E415
:101750009216D1F59F01220F331F220F331FF9017B
:10176000E40FF51F80911A0190911B01892F992791
:1017700083A780911A0190911B0184A780910E018B
:1017800090910F01892F992785A780910E01909143
:101790000F0186A7112309F441C000E0F901349735
:1017A0001E161F06DCF520E2BF01DA01A00FB11DF5
:1017B000FD0183A5882309F423A70F5F802F9927B4
:1017C0008617970794F32AC09F012E0F3F1FF90138
:1017D000E40FF51F80910E0190910F01892F992739
:1017E00083A780910E0190910F0184A71123B1F07E
:1017F00000E0F90132971E161F0684F420E2BF01B3
:10180000DA01A00FB11DFD0183A5882309F423A7E8
:101810000F5F802F99278617970794F3112331F4D0
:10182000F1E0C454DF4FF883CC5BD040C554DF4FA8
:10183000A882CB5BD040C654DF4F1883CA5BD04030
:1018400054C9133009F451C9143009F04EC921E4C8
:10185000921609F04AC980910E0190910F01F6E0AD
:1018600096958795FA95E1F7EFE32E2E2822C0543E
:10187000DF4F3881C05CD040321509F436C9C054FE
:10188000DF4F2882C05CD04060901A0170901B012D
:101890007694679480911C0190911D01AA27BB2723
:1018A00083709070A070B0706FE0880F991FAA1FAE
:1018B000BB1F6A95D1F7680E791E20910E013091F9
:1018C0000F01232F332722952F7080911A019091B9
:1018D0001B018170907044E0880F991F4A95E1F7D1
:1018E000280FC154DF4F2883CF5BD04040900E01BA
:1018F00050900F016FE14622552480910E01909186
:101900000F0185FF07C07DE2CF53DF4F7883C15CB5
:10191000D04006C08BE2CF53DF4F8883C15CD040FC
:101920008EE190E0489ED001499EB00D589EB00DCA
:1019300011242D0180910E0190910F019F938F939F
:1019400080911A0190911B019F938F9380911C01AC
:1019500090911D01837090709F938F938AE795E01B
:101960009F938F930E94AB0E6301EE24D7FCE0940B
:10197000FE2CC701B6010E949B1377FE06C020E033
:1019800030E040E857E40E94F6122DEC38E94BE6CF
:1019900056E40E94F512DC01CB0120E030EA46EB70
:1019A00053E4BC01CD010E943813DC01CB01BC0122
:1019B000CD010E94A513DC01CB01BC01CD010E9429
:1019C0007E134B015C01C354DF4F79836883CD5B89
:1019D000D040C701B6010E949B1377FE06C020E0ED
:1019E00030E040E857E40E94F61226E630EB49E684
:1019F00056E40E94F5126B017C01C354DF4F6881ED
:101A00007981CD5BD040882777FD8095982FCE5384
:101A1000DF4F688379838A839B83C25CD0400E94B6
:101A20009B1397FE06C020E030E040E857E40E9498
:101A3000F61220E030EA46EB53E40E940C14DC017D
:101A4000CB01BC01CD010E94A513DC01CB019C019F
:101A5000AD01C701B6010E94F512DC01CB0121E006
:101A60003DEC44EF51E4BC01CD010E943813DC0190
:101A7000CB01BC01CD010E94A513DC01CB01BC014F
:101A8000CD010E947E13DC01CB01382E83010C5660
:101A90001A43C801AA2797FDA095BA2FBC01CD0112
:101AA0000E949B136B017C018DB79EB708960FB601
:101AB000F8949EBF0FBE8DBF17FF0AC020E030E034
:101AC00040E857E4C701B6010E94F6126B017C01A1
:101AD000CE53DF4F688179818A819B81C25CD0407F
:101AE0000E949B1397FE06C020E030E040E857E4D8
:101AF0000E94F61220E030EA46EB53E40E940C14F8
:101B0000DC01CB01BC01CD010E94A513DC01CB019E
:101B10009C01AD01C701B6010E94F5127B018C0149
:101B2000832D9927AA2797FDA095BA2FBC01CD0137
:101B30000E949B13DC01CB0121E03DEC44EF51E41A
:101B4000BC01CD010E940C14DC01CB01BC01CD0114
:101B50000E94A513DC01CB019C01AD01C801B701B6
:101B60000E94F512DC01CB01BC01CD010E947E1365
:101B7000DC01CB01482F832D8E50823010F401E020
:101B800001C000E0202F3327C354DF4FE881F981E3
:101B9000CD5BD040E20FF31FE459F84F84EF9FEF85
:101BA000289FD001299FB00D389FB00D1124232DFF
:101BB0002A0F2150C2016CE370E00E9454146C01A2
:101BC0009F938F93C2016CE370E00E9454147B01D9
:101BD0007F936F93CF53DF4FB881C15CD0408B2F81
:101BE00099279F938F93822D99279F938F93C15409
:101BF000DF4F3881CF5BD040832F99279F938F93FE
:101C00007F926F92842F99279F938F93822F99278A
:101C10009F938F93FF93EF938FE895E09F938F931C
:101C20000E94AB0E6DB77EB76C5E7F4F0FB6F89417
:101C30007EBF0FBE6DBFCF53DF4F7881C15CD040F8
:101C40007D3249F4C154DF4F2881CF5BD0402E193B
:101C5000822D8C1911C0C2016CE370E00E945414F3
:101C6000C154DF4F2881CF5BD040260FC2016CE307
:101C700070E00E945414820D87FF02C0845C2150E2
:101C80008C3314F08C532F5F27FD285E28310CF025
:101C90002851992787FD90959F938F93822F99279D
:101CA00087FD90959F938F9386EC95E09F938F93FC
:101CB0000E94AB0E8DB79EB706960FB6F8949EBFE6
:101CC0000FBE8DBF0C9475050F931F93CF93DF93B9
:101CD0008C01EB01009711F4672BC1F16EE070E00D
:101CE00081E090E00E948D11FC01892B71F180E868
:101CF0008383209771F0D387C28781E883838091A3
:101D0000250190912601892B21F4F0932601E0937F
:101D1000250101151105C9F01187008783818260B3
:101D200083838091270190912801892B71F4F0938E
:101D30002801E09327018091290190912A01892BA4
:101D400021F4F0932A01E0932901CF01DF91CF9193
:101D50001F910F910895CF93DF93CDB7DEB745E084
:101D600050E04C0F5D1FFA0121913191AF01A0911C
:101D70002701B0912801FD01838188608383B90127
:101D800080912701909128010E94D00EE0912701B7
:101D9000F09128012381277F2383DF91CF9108953C
:101DA0002F923F924F925F926F927F928F929F926B
:101DB000AF92BF92CF92DF92EF92FF920F931F9359
:101DC000CF93DF93CDB7DEB762970FB6F894DEBF3F
:101DD0000FBECDBFEE24FF2487011C017E876D87D7
:101DE0002A01CC24DD24FC01D782C682838181FDB7
:101DF00068C28FEF9FEF78C28D859E8501969E8782
:101E00008D87C0FE4BC28F8580538A30D0F49F856A
:101E1000903339F4662029F4C3FC03C0E0E0F1E01C
:101E20008DC08AE0689E602C1124FF856F0E20ED26
:101E3000620E67FE02C05FE7652EC3FC42C2762CCD
:101E400040C2C3FE04C0662011F441E0642EEF8559
:101E50008E2F992787FD9095883691058CF58536CC
:101E600091050CF06EC08335910509F493C084355B
:101E70009105CCF48B32910509F449C08C3291055F
:101E80004CF48032910509F446C08332910509F47F
:101E90004AC0FEC18D32910509F440C08E329105D1
:101EA00009F444C0F5C18336910509F450C0843665
:101EB00091050CF08AC08835910509F4BCC0E8C1D1
:101EC0008037910509F4B1C08137910584F48C36CF
:101ED000910591F18D3691052CF48936910509F41F
:101EE00074C0D6C18F36910509F49CC0D1C1853725
:101EF000910509F4A2C08637910524F48337910532
:101F000071F1C6C18837910509F495C0C1C180E15E
:101F100090E0C82AD92AE0E2F0E010C080E890E022
:101F2000C82AD92ACEC1E0E4F0E008C088E090E0F9
:101F3000C82AD92A6624C5C1E4E0F0E0CE2ADF2A07
:101F4000C0C13FE3E32E7A94F3E6FF873CC1F20180
:101F500082E090E0480E591EE0807A9434C1F2018C
:101F600082E090E0480E591EA081B1817D01C3FE40
:101F700009C0862D992787FD9095BC01CD010E944F
:101F8000BD121FC0FD0101900020E9F73197EA1B47
:101F9000E88B18C0F20182E090E0480E591E0190D3
:101FA000F081E02D7F01C3FE09C0862D992787FDB2
:101FB0009095BC01CF010E94A81203C0CF010E94DE
:101FC0009F12888B9889791AFEC0C2FE0AC0F2015E
:101FD00084E090E0480E591E208131814281538176
:101FE0000CC0F20182E090E0480E591E8081918180
:101FF0009C01442737FD4095542F79018A0157FFF2
:102000000CC0E2E0F0E0CE2ADF2A10950095F094B3
:10201000E094E11CF11C011D111D8FEB9FEFC82204
:10202000D92227C098E0988B08C0E0E4F0E0CE2ADF
:10203000DF2AF8E7FF8720E1288BC2FE0AC0F20101
:1020400084E090E0480E591E208131814281538105
:102050000AC0F20182E090E0480E591E8081918111
:102060009C014427552779018A01EFECFFEFCE222E
:10207000DF22CE0101969A8B898B9889892E99242B
:10208000AA24BB24C801B701A50194010E946814C9
:10209000DC01CB01E989FA8980838A3024F0FF854D
:1020A0008F0F815201C0805DE989FA898193FA8B93
:1020B000E98BC801B701A50194010E946814790158
:1020C0008A012115310541055105E1F6E98881E0D4
:1020D00090E08C0F9D1FE81AC60182739070892BC7
:1020E00009F07A94C6FE0DC0872D992787FD90953B
:1020F000E889E03121F42EEF722E780E02C0782E9E
:102100007A94C3FE0FC0262D332727FD30958E2DE0
:102110009927821793072CF087EF9FEFC822D922C7
:1021200001C06E18C3FE02C0761801C07E18C60139
:1021300080789170892B51F4872D7A94181634F495
:10214000B10180E290E00E94C812F6CFC1FE04C047
:10215000B1018DE290E00BC0C4FE04C0B1018BE27E
:1021600090E005C0C5FE05C0B10180E290E00E948C
:10217000C812C6FE10C0B10180E390E00E94C812F0
:102180009889903141F4B101EF858E2F992787FD11
:1021900090950E94C812D0FE0AC0872D7A94181616
:1021A00034F4B10180E390E00E94C812F6CFC3FE80
:1021B0000AC0862D6A94181634F4B10180E390E0C9
:1021C0000E94C812F6CF90E8B92EBC2051F4872D9A
:1021D0007A94181634F4B10180E290E00E94C8129B
:1021E000F6CFFF85F33641F48E2DB101992787FD97
:1021F00090950E94C81240C02F852337B1F488897A
:102200008150888B8F3FC1F1F70180810894E11CD8
:10221000F11CB101992787FD90950E94C8129889F9
:102220009150988B9F3F81F727C0EF85E33579F474
:10223000F889F150F88BFF3FF9F0F7018491B10173
:1022400099270E94C8120894E11CF11CF1CF6E017D
:102250000894C11CD11C89899A898C159D0561F04F
:10226000E989FA898291FA8BE98BB101992787FD77
:1022700090950E94C812EFCFBB2069F0872D7A9409
:1022800018164CF4B10180E290E00E94C812F6CF1B
:10229000B1010E94C812CC24DD2413C09F85953261
:1022A00041F481E0C82ED12C6624762CEAE0E88B3C
:1022B00008C0B101FF858F2F992787FD90950E9457
:1022C000C812F101838183FF04C0ED85FE85F4917E
:1022D00003C0ED85FE85F081FF872F85222309F05D
:1022E0008BCDF1018681978162960FB6F894DEBF9F
:1022F0000FBECDBFDF91CF911F910F91FF90EF9057
:10230000DF90CF90BF90AF909F908F907F906F9015
:102310005F904F903F902F9008950F931F93CF930E
:10232000DF93869F8001879F100D969F100D1124CB
:10233000C8010E94A911EC01009729F0A80160E0F2
:1023400070E00E94B312CE01DF91CF911F910F91E7
:102350000895CF93DF93AC01029710F442E050E070
:1023600020E030E0A0912D01B0912E01BD01F901D6
:10237000109709F44CC08D919C9111978417950783
:1023800031F14817590738F42115310519F0821732
:10239000930708F49C01FD01A281B381109759F7BE
:1023A00021153105A1F1C901841B950B049708F48F
:1023B000A901DB01E0E0F0E0109749F18D919C91DB
:1023C000119782179307F9F44217530779F4ED0137
:1023D0008A819B81309719F09383828304C0909304
:1023E0002E0180932D01CD0102964AC0241B350B8E
:1023F000FD01E20FF31F41935193225030402D9382
:102400003C93CF013DC0FD01A281B381D5CF809126
:102410002B0190912C01892B41F480910201909124
:10242000030190932C0180932B01E0910001F09126
:102430000101309741F4EDB7FEB78091040190910E
:102440000501E81BF90BA0912B01B0912C019F0114
:102450002A1B3B0B2417350788F0CA010296281760
:10246000390760F0CD01840F951F029690932C01DF
:1024700080932B014D935D93CD0102C080E090E0ED
:10248000DF91CF910895CF93DF93009709F454C063
:10249000DC011297ED011B821A8280912D0190912F
:1024A0002E01009721F1FC0140E050E0EA17FB0704
:1024B00018F1ED01FB83EA832D913C911197C20F36
:1024C000D31FCE0102968E179F0771F48A819B81DC
:1024D000280F391F2E5F3F4F11963C932E93828118
:1024E0009381FD01938382834115510559F4B09383
:1024F0002E01A0932D0120C0AF010280F381E02DB9
:102500003097A1F6EA01BB83AA83CA01029628810B
:102510003981820F931F8A179B0771F48D919C91CB
:102520001197280F391F2E5F3F4F39832883FD01F4
:10253000828193819B838A83DF91CF910895FC01EF
:1025400005900020E9F7809590958E0F9F1F0895C4
:10255000FC010590615070400110D8F7809590956E
:102560008E0F9F1F0895DC0140FF03C001C06D93D3
:102570006D9342505040D8F70895FC01615070406F
:1025800001900110D8F7809590958E0F9F1F0895A8
:102590000F931F93CF93DF938C01EB018B819927CE
:1025A00081FF1CC082FF0DC02E813F818C819D81E7
:1025B0002817390764F4E881F9810193F983E883E6
:1025C00006C0E885F985802F0995892B39F48E811D
:1025D0009F8101969F838E83C80102C08FEF9FEF7A
:1025E000DF91CF911F910F9108955058192EE6D089
:1025F00001D0C9C0BA176207730784079507B1F104
:1026000088F40EF410940B2EBA2FA02D062E622FF4
:10261000202D072E732F302D082E842F402D092EAC
:10262000952F502DFF275523B9F0591B49F0573EE0
:1026300098F0469537952795A795F0405395C9F79B
:1026400076F0BA0F621F731F841F30F48795779559
:102650006795B795F040939517FA0F2E0895BF1B15
:10266000BB27BA0B620B730B840BF6CFDEF6D2C01E
:10267000A5D001D088C0552359F0992369F09F5700
:102680005F57951B33F442F4903811F4915805C00C
:1026900092C091589F3F09F4BDC0BB271124621717
:1026A0007307840730F4660F771F881FBB1F915094
:1026B00098F311D00F920FD00F920DD0A0E82617EB
:1026C000370748071B0609F0A048BA2F602D7F91F5
:1026D0008F9100240895A0E80024621773078407EF
:1026E000B10528F0621B730B840BB1090A2A660F2F
:1026F000771F881FBB1FA69581F7089597FB6AD0A7
:102700009F3738F0FEE9F91B982F872F762F6B2F14
:1027100005C07DC09695879577956795F150D0F760
:102720003EF490958095709561957F4F8F4F9F4FA8
:102730000895E89403C097FB0EF4F3DFB62F672FDC
:10274000782F892F9EE900241EC052D09F3760F455
:102750000EF05DC09FEB80E8772766270895869589
:1027600077956795B11D93959639C8F32EF4BB23E1
:1027700019F06F5F7F4F8F4FBB2705C09A95BB0F36
:10278000661F771F881F11249923A1F08823B2F7B1
:102790009F3F59F0BB0F48F421F4002011F460FF73
:1027A00004C06F5F7F4F8F4F9F4F881F979587950E
:1027B00097F908952CC09FEF80EC0895052E092607
:1027C00007FA440F551F5F3F79F0AA27A51708F0B5
:1027D00051E04795880F991F9F3F31F0BB27B917EC
:1027E00008F091E0879508959F919F911124E3CF80
:1027F00097FB880F991F9F3F31F0BB27B91708F04F
:1028000091E0879508959F919F911124D4CF6627D9
:102810007727882799270895D1DF01D0B4CF99234E
:1028200039F0552329F09F575F57950F13F49AF10C
:10283000F1CF91589F3FE1F3629FA12D0F92BB27EB
:10284000639FA00DB11DEE27729FA00DB11DEE1F5D
:10285000AF93AA27649FB00DE11D739FB00DE11DDA
:10286000AA1F6627829FB00DE11DA61F5527749FE2
:10287000E00DA11D551F839FE00DA11D561F849FD4
:10288000A00D511D852F7A2F6E2F1F900F9088233A
:102890001AF4939539F48FCF000C111CBB1F661FDF
:1028A000771F881F01280895AA1BBB1B51E107C091
:1028B000AA1FBB1FA617B70710F0A61BB70B881FD0
:1028C000991F5A95A9F780959095BC01CD0108955F
:1028D000A1E21A2EAA1BBB1BFD010DC0AA1FBB1F24
:1028E000EE1FFF1FA217B307E407F50720F0A21B96
:1028F000B30BE40BF50B661F771F881F991F1A9403
:1029000069F760957095809590959B01AC01BD012C
:04291000CF01089556
:0629140000002F0120006D
:00000001FF
